:020000040800F2
:10000000E80C00202D020008FF1200085912000819
:10001000FD1200081D040008111E00080000000069
:10002000000000000000000000000000451400086F
:100030007104000800000000011300080F150008FB
:10004000470200084702000847020008470200086C
:10005000470200084702000847020008470200085C
:10006000470200084702000847020008470200084C
:10007000470200084702000847020008470200083C
:10008000470200084702000847020008470200082C
:10009000470200084702000847020008470200081C
:1000A00047020008751600084702000847020008CA
:1000B000C51600080000000000000000470200080C
:1000C00047020008470200084702000847020008EC
:1000D000470200085919000847020008A51900083E
:1000E0007304000847020008000000000000000040
:1000F0000000000000000000000000000000000000
:10010000000000004702000800000000470200084D
:10011000000000000000000047020008470200083D
:10012000470200084702000847020008470200088B
:10013000470200080000000000000000000000006E
:10014000470200084702000847020008470200086B
:10015000470200084702000847020008470200085B
:10016000470200084702000847020008000000009C
:10017000470200084702000847020008000000008C
:1001800047020008470200084702000800F002F892
:1001900000F03CF80AA090E8000C82448344AAF1E5
:1001A0000107DA4501D100F031F8AFF2090EBAE8E3
:1001B0000F0013F0010F18BFFB1A43F0010318479B
:1001C0005C2700007C270000103A24BF78C878C163
:1001D000FAD8520724BF30C830C144BF04680C604D
:1001E000704700000023002400250026103A28BF95
:1001F00078C1FBD8520728BF30C148BF0B60704799
:100200001FB502F0E6F81FBD10B510BD00F08AF86A
:100210001146FFF7F5FF01F051FF00F0A8F803B415
:10022000FFF7F2FF03BC00F0AFF800000948804779
:1002300009480047FEE7FEE7FEE7FEE7FEE7FEE7C8
:10024000FEE7FEE7FEE7FEE704480549054A064BE0
:10025000704700009D1500088D010008E806002089
:10026000E80C0020E8080020E808002010B5203A3B
:10027000C0F00B80B1E81850203AA0E81850B1E85F
:100280001850A0E81850BFF4F5AF5FEA027C24BF15
:10029000B1E81850A0E8185044BF18C918C0BDE80C
:1002A00010405FEA827C24BF51F8043B40F8043BD5
:1002B00008BF7047D20728BF31F8023B48BF11F88A
:1002C000012B28BF20F8023B48BF00F8012B7047E4
:1002D0004FF0000200B5134694469646203922BFDF
:1002E000A0E80C50A0E80C50B1F12001BFF4F7AF2A
:1002F000090728BFA0E80C5048BF0CC05DF804EB0C
:10030000890028BF40F8042B08BF704748BF20F879
:10031000022B11F0804F18BF00F8012B7047704777
:1003200070477047754600F02BF8AE4605006946E9
:10033000534620F00700854618B020B5FFF784FF2C
:10034000BDE820404FF000064FF000074FF00008D6
:100350004FF0000B21F00701AC46ACE8C009ACE857
:10036000C009ACE8C009ACE8C0098D46704710B5BB
:100370000446AFF300802046BDE81040FFF74FBFB2
:10038000004870478406002001491820ABBEFEE7F4
:100390002600020070470000F8B50025009501F026
:1003A00073FB1C4C94F86802012810D194F8B40235
:1003B0000126194F01280BD002281CD084F868525E
:1003C000C4F86452257084F8AD5287F82460F8BDF3
:1003D00094F8B502012804D1A079342801D101F0A4
:1003E000D1FE84F86852C4F86452257084F8AD5286
:1003F00087F82460F8BDA079342801D100F03EF8D8
:1004000084F86852C4F86452257084F8AD5287F8B5
:100410002460F8BDA402002014000020FEE70000C4
:1004200000B5AFB06422104916A8FFF71FFF0020E7
:100430000E4916AA01EB800393ED000A02EB80033C
:1004400083ED000A401CC0B21928F3D354221AA924
:100450006846FFF70BFF16A80FC800F00BF901F074
:1004600031FA2FB000BD0000B82800087405002044
:1004700070474FF4806000F05DB9000010B54B4943
:100480000879402849D0412846D10020484A0B1815
:100490001418DB7984F83030401CC0B20C28F6D335
:1004A00000200B181418DB7C2372401CC0B20428F7
:1004B000F7D300200B181418DB7D84F83C30401C67
:1004C000C0B20828F6D300200B181418DB7F237362
:1004D000401CC0B20428F7D300200B18141893F85E
:1004E000233084F84430401CC0B20828F5D30020E3
:1004F0000B18141893F82B302374401CC0B2042836
:10050000F6D300200B18141893F82F3084F84C30D1
:10051000401CC0B21428F5D310BD0020254A0B188A
:100520001418DB7984F83030401CC0B20C28F6D3A4
:1005300000200B181418DB7C2372401CC0B2042866
:10054000F7D300200B181418DB7D84F83C30401CD6
:10055000C0B20828F6D300200B181418DB7F2373D1
:10056000401CC0B20428F7D300200B18141893F8CD
:10057000233084F84430401CC0B20828F5D3002052
:100580000B18141893F82B302374401CC0B20428A5
:10059000F6D300200B18141893F82F3084F84C3041
:1005A000401CC0B21428F5D310BD0000A4020020E6
:1005B000D8050020740500202DE9F0412C4D0024C1
:1005C0002846A97D90F82400002942D00227012660
:1005D000B0B195F8260010B1012811D108E0012032
:1005E00000F031FF2435AE702C7105F8244907E086
:1005F000022000F028FF2435AF702C7105F8244943
:1006000095F82500B0B195F8270010B1012811D157
:1006100008E0032000F017FF2535AE702C7105F8B7
:10062000254907E0042000F00EFF2535AF702C713E
:1006300005F8254995F82600022808D195F82700E5
:10064000022804D105F8164F2C746C742E75BDE881
:10065000F08195F82A100029F9D00028F7D095F8F4
:1006600025000028F3D0FFF7DBFE85F82A40EEE7EF
:10067000140000200FB410B5ADF5127D0FA801F0E5
:10068000BDFC9DED960ADDED970A9DED981A9DED56
:10069000A02A9DEDA13ADDEDA23ADDEDA32A9DED64
:1006A000A44ADDEDA54ADDEDA61A9DEDA75ADDEDC4
:1006B000A85A9DEDA96ADDEDAA6A9DEDAB7A8DED94
:1006C000002A8DED013ACDED023A8DED030ACDED14
:1006D000042A8DED054ACDED060ACDED074ACDED94
:1006E000081A8DED091A8DED0A5ACDED0B5A8DEDD4
:1006F0000C6ACDED0D6A8DED0E7A0FA9684601F0FA
:1007000089FB012800D14124022800D1422403287A
:1007100000D14324042800D14424052800D14524D5
:10072000401C00D146240DF5127D204610BC5DF81A
:1007300014FB704710B504490A68024202D00860F1
:10074000FFF7F7FF10BD0000140401402DE9F84F3A
:100750000022DFF860A14FF003084FF00F090AF103
:10076000040BA0E0012595402B40002B71D04C6874
:10077000012C05D0022C03D0112C01D0122C10D149
:100780008668540008FA04F7BE43CF68A740374391
:1007900087604468AC430D79C5F300159540254347
:1007A0004560C468570008FA07F5AC438E68BE4040
:1007B0002643C6604C68022C01D0122C12D1D408FA
:1007C00000EB840CDCF820605407E40E09FA04FE08
:1007D00026EA0E06D1F810E00EFA04FE4EEA060EE6
:1007E000CCF820E00468AC430D7905F00305BD406A
:1007F000254305604C68E40054D52F4C256E45F028
:1008000001052566246E04F0010400942B4C22F0AF
:1008100003052E19B7689407250F09FA05F4A743B5
:10082000B0F1904F04D0264CA04203D1012412E035
:10083000002410E0234CA04201D102240BE0224C02
:10084000A04201D1032406E0204CA04202D104249E
:1008500001E027E00724AC403C43B460DAF80040F4
:100860009C434D68ED0300D51C43CAF80040DBF8FB
:1008700000409C434D68AD0300D51C43CBF80040BD
:100880000C4D08352C689C434E68F60200D51C437D
:100890002C60084D0C352C689C434E68B60200D580
:1008A0001C432C60521C0B6833FA02F47FF45AAFDD
:1008B00000F00EB8000401400010024000000140AA
:1008C0000004004800080048000C004800100048E0
:1008D00018BCBDE8E08F002A01D0816170478162B9
:1008E0007047000001488068704700000000002049
:1008F000024881684268114481607047000000200E
:1009000010B50024032000F067F8002000F008F87C
:1009100008B1012401E000F029F8204610BD0000D4
:1009200070B5054600240F4E7068002817D04FF4AC
:100930007A71B1FBF0F00C490968B1FBF0F000F0FE
:1009400077FC08B101240BE0102D06D200222946C5
:10095000501E00F021F8356002E0012400E001247F
:10096000204670BD000000200C00002008B509489A
:10097000016E41F001010166016E01F0010100917B
:10098000816D41F080518165806D00F08050009054
:1009900008BD000000100240F0B40D460D4B1B686E
:1009A000C3F30223C3F10704042C00D90424191D46
:1009B000072901D2002300E0DB1E012606FA04F11C
:1009C000491E294099409E40761E16403143F0BC96
:1009D00001F096BA0CED00E000F00701054A10683E
:1009E0004FF6FF03184040EA012003490843106016
:1009F000704700000CED00E00000FA051749B0F563
:100A0000007F0CD00868C0F34120022805D0086898
:100A100020F4C06040F480600860002070470868DF
:100A2000C0F341200128F8D0086820F4C06040F4E9
:100A3000007008600A48322200685043094AB0FB3F
:100A4000F2F0401C00E0401E4A69520501D5002822
:100A5000F9D148694005E0D5032070470070004097
:100A60000C00002040420F000248006800F4C06003
:100A700070470000007000402DE9F04704460D4625
:100A8000002C17D0DFF82481D8F8000000F0070010
:100A9000A84211D2D8F8000020F007002843C8F877
:100AA0000000D8F8000000F00700A84204D00120A0
:100AB000BDE8F0870120FBE720783D4EC00732D02B
:100AC0006068032807D002280AD070B13168490550
:100AD00010D40120ECE7316889010BD40120E7E74D
:100AE0003168890306D40120E2E73168890701D41F
:100AF0000120DDE7B16821F003010143B160FFF798
:100B0000F1FE074641F2883906E0FFF7EBFEC01B15
:100B1000484501D90320CBE7B068616800F00C00BC
:100B2000B0EB810FF1D12078800705D5B068A168BE
:100B300020F0F0000843B060D8F8000000F0070093
:100B4000A8420ED9D8F8000020F007002843C8F8C2
:100B50000000D8F8000000F00700A84201D00120F2
:100B6000A6E72078400705D5B068E16820F4E0608A
:100B70000843B0602078000706D5B068216920F4EA
:100B8000605040EAC100B06000F01AF8B168094A4C
:100B9000C1F30311515C01F01F01C8400649086010
:100BA00006480068BDE8F047FFF7BABE00200240E3
:100BB00000100240E82300080C0000200000002084
:100BC00070B500220020244B996801F00C01DC680C
:100BD00004F00304214D6E10002908D00C2901D126
:100BE000012C04D0042913D0082913D013E01A686B
:100BF000120704D4D3F89420C2F3032202E01A6847
:100C0000C2F30312164C54F8222021B9104602E018
:100C1000284600E030460C2918D1D86800F00300BF
:100C2000022814D0032814D01046D968C1F3021149
:100C3000491CDA68C2F306224243B2FBF1F0D968DC
:100C4000C1F34161491C4900B0FBF1F070BD284679
:100C5000EBE73046E9E70000001002400024F40012
:100C6000F82300082DE9F8430446002C0DD0F94E76
:100C7000B06800F00C05F06800F003072078C006AB
:100C80006AD595B10C2D03D004E00120BDE8F883AE
:100C9000012F0AD0A06900287DD0306840F0010003
:100CA0003060FFF71FFE80465FE03068800701D5A7
:100CB000A06938B1206A3168090705D5316801F0AB
:100CC000F00106E00120E1E7D6F8941001F470612C
:100CD0000909884216D900F073FB08B10120D5E755
:100CE000306840F0080030603068216A20F0F00081
:100CF000084330607068E16920F47F4040EA0120D9
:100D0000706017E0306840F0080030603068216A99
:100D100020F0F000084330607068E16920F47F4003
:100D200040EA012070602DB9206A00F049FB08B14B
:100D30000120ABE7FFF744FFB168C74AC1F30311D5
:100D4000515C01F01F01C840C4490860C4480068F4
:100D5000FFF7E6FD002899D130E0FFF7C3FDA0EBD7
:100D60000800022801D9032090E730688007F4D5F5
:100D7000306840F0080030603068216A20F0F000F0
:100D8000084330607068E16920F47F4040EA012048
:100D9000706013E0FFE7306820F001003060FFF77B
:100DA000A1FD804607E0FFF79DFDA0EB08000228AB
:100DB00001D903206AE730688007F4D42078C0079F
:100DC0004AD0082D18D00C2D01D1032F14D0606803
:100DD000B0F5803F17D0B0F5A02F19D0306820F4BF
:100DE00080303060306820F480203060606820B34C
:100DF000FFF778FD80461CE0306880032CD56068E2
:100E000050BB012042E7306840F480303060EDE7AD
:100E1000306840F480203060306840F480303060CA
:100E2000E4E7FFF75FFDA0EB0800642801D9032089
:100E30002CE730688003F4D50EE0FFF753FD8046C1
:100E400007E0FFF74FFDA0EB0800642801D903205D
:100E50001CE730688003F4D42078800742D5042D45
:100E60000DD00C2D01D1022F09D0E06840B33068BD
:100E700040F480703060FFF735FD074615E03068BC
:100E8000400501D5E06838B17068217C20F0F85049
:100E900040EA0160706025E00120F7E6FFF722FDDF
:100EA000C01B022801D90320F0E630684005F5D5C3
:100EB0007068217C20F0F85040EA0160706011E019
:100EC000306820F480703060FFF70CFD074606E0C4
:100ED000FFF708FDC01B022801D90320D6E63068C1
:100EE0004005F5D4207800072CD56069A8B1D6F864
:100EF000940040F00100C6F89400FFF7F3FC0746A9
:100F000006E0FFF7EFFCC01B022801D90320BDE675
:100F1000D6F894008007F4D514E0D6F8940020F0B9
:100F20000100C6F89400FFF7DDFC074606E0FFF776
:100F3000D9FCC01B022801D90320A7E6D6F89400EB
:100F40008007F4D42078400774D54FF00008B06DC6
:100F5000C00009D4B06D40F08050B065B06D00F0B5
:100F6000805000904FF00108DFF8F890D9F80000A9
:100F7000C00514D4D9F8000040F48070C9F800000E
:100F8000FFF7B0FC074606E0FFF7ACFCC01B0228E9
:100F900001D903207AE6D9F80000C005F4D5A0688D
:100FA000012813D0052818D056F8900F20F0010022
:100FB0003060306820F0040046F89009A06841F2E3
:100FC000883908B3FFF78EFC074618E0D6F8900082
:100FD00040F00100C6F89000F0E756F8900F40F09E
:100FE00004003060306840F0010046F89009E5E701
:100FF000FFF778FCC01B484501D9032046E6D6F828
:1010000090008007F4D50EE0FFF76CFC074606E081
:10101000FFF768FCC01B484501D9032036E6D6F827
:1010200090008007F4D4B8F1010F03D1B06D20F027
:101030008050B0652078800637D5606A00B3D6F856
:10104000980040F00100C6F89800FFF74BFC0746F7
:1010500011E0000000100240E82300080C0000200E
:101060000000002000700040FFF73CFCC01B02287D
:1010700001D903200AE6D6F898008007F4D514E0D9
:10108000D6F8980020F00100C6F89800FFF72AFC77
:10109000074606E0FFF726FCC01B022801D9032003
:1010A000F4E5D6F898008007F4D4A06AE8B30228E3
:1010B00014D00C2D7ED0306820F080703060306805
:1010C000000103D4F06820F00300F060F068564996
:1010D0000840F060FFF706FC04469EE0F068E26A14
:1010E00000F003014FF0FF37914226D1216B00F051
:1010F0007002491EB2EB011F1FD1626B00F4FE416A
:10110000B1EB022F19D194F8382000F07841B1EBFF
:10111000C26F12D1A28F00F4C00107EB5202B1EBF3
:10112000425F0AD100F0C06000E06EE094F8401029
:1011300007EB5101B0EB416F4ED00C2D4AD0306817
:10114000400101D50120A1E5306820F080703060B9
:10115000FFF7C8FB054606E0FFF7C4FB401B02286B
:1011600001D9032092E530688001F5D454F82C1F92
:101170006068228A401E41EA0010A16807EB520213
:10118000090241EA42510843217D07EB510140EA3F
:101190004160217B40EAC160F168244A1140084364
:1011A000F060306840F080703060F06840F080702F
:1011B000F06000E036E0FFF795FB044606E0FFF73D
:1011C00091FB001B022801D903205FE530688001F4
:1011D000F5D525E0012059E53068800120D430683C
:1011E00040F080703060F06840F08070F060FFF791
:1011F00079FB044606E0FFF775FB001B022801D9C6
:10120000032043E530688001F5D509E0FFF76AFB6C
:10121000001B022801D9032038E530688001F5D48D
:10122000002033E5012031E5FFFFEEFE8C809D01BB
:1012300010B5401EB0F1807F01D3012010BD4FF0EA
:10124000E02460610F21601700F05AFE0020A061C9
:1012500007202061002010BDFEE7000000B587B028
:10126000142102A8FFF734F80B48C16C41F00401C7
:10127000C164C06C00F0040001904FF480500290F3
:101280000120039004900220059002A90348FFF773
:101290005DFA07B000BD00000010024000080048E1
:1012A00000B587B0142102A8FFF712F80B48C16CF3
:1012B00041F00201C164C06C00F0020001904FF4E3
:1012C000807002900120039004900220059002A9F2
:1012D0000348FFF73BFA07B000BD000000100240D2
:1012E0000004004804490A798A703422CA704022F6
:1012F0000A71487170470000A4020020FEE7FEE773
:10130000704743780278934201D100207047C31C94
:10131000D25C0A7001784FF41872491CB1FBF2F3E9
:1013200002FB1311017001207047000030B587B037
:10133000142102A8FEF7CCFF0E48C16C41F0040155
:10134000C164C06C00F0040001904FF400440294AA
:1013500001200390049000200590074D02A9284623
:10136000FFF7F4F9002221462846FFF7B4FA07B048
:1013700030BD000000100240000800480122D103E7
:101380000148FFF7A8BA00000008004830B54278CD
:101390004FF418731446521CB2FBF3F503FB1522ED
:1013A0000578AA4201D1002030BDC21CA154417869
:1013B000491CB1FBF3F203FB12114170012030BD57
:1013C000F8B5054600241D4EB06DC00002D5FFF7EC
:1013D0004BFB0DE0B06D40F08050B065B06D00F09B
:1013E00080500090FFF740FBB16D21F08051B16556
:1013F000B0F5007F04D0802D0AD94FF003040DE032
:10140000802D0BD9A02D01D9022407E0012405E08D
:1014100001D1022402E0702D00D1012408480168A6
:1014200021F0070121430160006800F00700A0429D
:1014300001D00120F8BD0020F8BD000000100240DE
:101440000020024070477CB50021009101910125E8
:10145000FF22AB2334210A24012819D002282ED0E0
:10146000AA2155221023032840D004280FD18DF83B
:1014700000108DF801208DF8023081208DF80300D6
:1014800090208DF804000521684600F0A7F97CBD86
:101490008DF800208DF801308DF8021040208DF875
:1014A00003008DF804408DF805508DF806103720A4
:1014B0008DF807000821684600F022FA7CBD8DF8FF
:1014C00000208DF801308DF8021041208DF80300C6
:1014D0008DF804408DF805508DF806109F208DF88A
:1014E00007000821684600F00BFA7CBD8DF800105B
:1014F0008DF801208DF8023080208DF803008F20B8
:101500008DF804000521684600F068F97CBDFFF7FE
:10151000EFB9000010B598B0442107A8FEF7D8FE37
:10152000142102A8FEF7D4FE1B48816D41F08051C2
:101530008165806D00F080500190012107910804C1
:1015400008900220119003241294139114211491F5
:10155000072115911690179007A8FFF783FB10B18C
:10156000012018B010BD0F200290039400200490B9
:101570004FF4A06105910690042102A8FFF77CFAC0
:1015800008B10120EDE74FF40070FFF737FA08B11A
:101590000120E6E70020E4E7001002400D48016862
:1015A00041F4700101600C48016841F001010160E3
:1015B000002181600268094B1A4002608214C260F7
:1015C000026822F48022026081610249C0038039EE
:1015D0000860704788ED00E000100240FFFFF6EA67
:1015E00010B5FFF78DF9FFF795FF502000F0D6FCFE
:1015F000FFF79CFEFFF7C2FE322000F0D5FC4FF44F
:101600006144204600F016F9204600F0EFF9312140
:1016100040F69F7000F0A2F8BDE81040092141F6A5
:101620003F7000F001B8000010B5104A136E43F48B
:10163000006313660E4A1060101D01600C48012102
:10164000143801600A481C38016841F0010101604A
:101650000021192000F064FC192000F037FC044838
:101660002838016841F00101016010BD00100240FE
:10167000282C014011480168C9071ED0016821F0DB
:10168000010101600E480188491C018002884FF465
:101690007A718A4200D301804188491C4180418887
:1016A00064290AD3002141808288521C828082886A
:1016B0000A2A02D38180012181757047102C0140D4
:1016C0001400002010B54FF080400169C9073FD0D9
:1016D000016921F0010101611E484189491C4181D4
:1016E0004189C82901D3C821418130F80C1F491C08
:1016F0000180017F491CC9B20177427F521CD2B2DE
:1017000042770C38012400233C2903D980F8283083
:1017100080F824403C2A03D980F8293080F82540FD
:101720008189C82903D38381018A491C0182C18B25
:1017300000290DD0491E89B2C183002908D106486D
:101740000178052904D00370C0F8643280F868324B
:1017500010BD000014000020A402002010B50B4AA8
:10176000936D43F00103936592049062D162D06857
:1017700040F00100D06001211C2000F0D1FB1C20B2
:1017800000F0A4FBBDE8104000F002B800100240D9
:101790004FF08040016841F0010101607047000096
:1017A00070B5044601220B4E150329463046FFF75B
:1017B00092F80A2000F006FC0748048006480C381E
:1017C00002685206FCD5002229463046FFF783F80E
:1017D000002070BD00080048284800402DE9F04175
:1017E00005460E460122DFF844801703394640467D
:1017F000FFF771F80A2000F0E5FB00220C480C4BC3
:101800000C3006E01C682406FCD5A95C0180521C43
:1018100092B2B242F6D318684006FCD5394640462B
:10182000BDE8F0410022FFF756B80000000800486C
:101830001C48004070B50546FFF732FD1D48C16CDD
:1018400041F00201C164016E41F4804101661A4C0D
:10185000206820F4A0402060206840F420402060F0
:1018600015482030016841F0EE41016013481449E9
:101870000068B0FBF5F0086011480D210C380160DC
:10188000016841F0200101600D48001F016841F02E
:10189000010101600321252000F052FB252000F00A
:1018A00022FB2046BDE8704000224FF48071FFF714
:1018B00012B8000000100240000400480C00002094
:1018C0000C38014070B5044601220B4E1502294622
:1018D0003046FFF700F80A2000F074FB0748048048
:1018E00006480C3802685206FCD5002229463046CC
:1018F000FEF7F1FF002070BD0004004828380140C9
:101900002DE9F04105460E460122DFF8448017021A
:1019100039464046FEF7DFFF0A2000F053FB002265
:101920000C480C4B0C3006E01C682406FCD5A95C66
:101930000180521C92B2B242F6D318684006FCD520
:1019400039464046BDE8F0410022FEF7C4BF000022
:10195000000400481C38014010B50F480468A00678
:1019600006D50D4808300088C1B20C48FFF70EFDBF
:101970000B48210703D5016841F008010160A10768
:1019800003D5016841F002010160610703D50168D8
:1019900041F00401016010BD1C38014040000020EE
:1019A0002038014010B50F480468A00605D50D4841
:1019B00008300088C0B200F083F90B48210703D536
:1019C000016841F008010160A10703D5016841F0F9
:1019D00002010160610703D5016841F00401016063
:1019E00010BD00001C4800402048004070B505466E
:1019F000FFF734FC1F48C16C41F00401C164816DE4
:101A000041F4802181651C4C206820F47000206026
:101A1000206840F42000206017482430016841F419
:101A2000EE4101601548164900688008B0FBF5F0EA
:101A3000086013480D210C380160016841F0200155
:101A400001600F48001F016841F00101016002219F
:101A5000272000F075FA272000F045FA00224FF405
:101A600080512046FEF737FF0649002081F83F00ED
:101A700070BD000000100240000800480C0000206B
:101A80000C4800403C0600202DE9F84F0027009745
:101A9000874E96F86802002822D16946A6F519708B
:101AA000FFF72FFC00281BD030780222814C4FF02A
:101AB00001084FF4FA75052812D2DFE800F003138D
:101AC0002F6198009DF80010AB2909D1D6F8640267
:101AD000421C3044C6F86422417086F80080E583D9
:101AE00000F0EAB89DF800000A2805D0AB280FD016
:101AF000C6F864723770F3E7D6F864124B1C3144B1
:101B0000C6F864324870327086F8B582E583E7E73C
:101B1000C6F8648286F80080E583E1E79DF800104E
:101B2000342912D0032240291AD0412918D0AB29D8
:101B300020D0D6F86402431C3044C6F864324170A9
:101B40003270E58386F8B482CAE7D6F86402431C93
:101B50003044C6F864324170E58386F8B422BFE7AA
:101B6000D6F86402431C3044C6F8643241703270C7
:101B7000E583B5E7C6F8648286F80080E583AFE7C1
:101B8000D6F864029DF80020411C3044C6F8641267
:101B9000427096F8B402042101280CD002289FD18B
:101BA000D6F8640205289BDB7279521D904297DBC0
:101BB0003170E58394E796F8B50202280CD001282D
:101BC0008ED1D6F8640204288ADB3279121D904245
:101BD00086DB3170E58383E7D6F8640205288ADB6B
:101BE0007279521D904286DB3170E58378E7D6F832
:101BF00064129DF80020481CC6F8640288194270DF
:101C000096F8B402DFF8A8904FF0050A09F106092A
:101C1000012813D0022897D17179701C491D00F05A
:101C2000A9F9717911F8091088423CD186F800A011
:101C300086F86882E58386F8AC7251E796F8B502BB
:101C4000022814D001288AD13179701C091D00F0B6
:101C500091F917493279491D515C88421ED186F8A5
:101C600000A086F86882E58386F8AC7238E771795F
:101C7000701C491D00F07EF9717911F80910884235
:101C800007D186F800A086F86882E58386F8AC72F2
:101C900026E73770C6F86472E78321E73770C6F825
:101CA0006472E7831CE73770C6F86472E78317E74E
:101CB000A40200201400002018BCBDE8E08F000042
:101CC000F0B5354A0023114692F83F600124AA2559
:101CD00091F83D10062E09D2DFE806F0030E210828
:101CE0003E51AA2803D002F83D3F9370F0BD3D322B
:101CF0009470AA311170F0BD5070552805D0AA28F3
:101D000009D03D3293701370F0BD02203D329070C7
:101D100055311170F0BD02F83D5F9470F0BD9070C8
:101D2000102809D080280BD0812809D0AA280FD0EC
:101D30003D3293701370F0BD103182F83D10F0BD4C
:101D4000042482F83F40084482F83D005372F0BDFD
:101D500002F83D5F9470F0BD0F49537A0A31585430
:101D6000517A491CC9B2517292F83D30184482F838
:101D70003D000829EFD3052082F83F00F0BD8142E5
:101D800005D0FF203D32507013709370F0BD0620D7
:101D90003E3250701370F0BD3C06002070B5184BF9
:101DA00093F83F00062829D193F83E000024FF282D
:101DB00007D098781349144A802805D0812816D175
:101DC0000CE083F83E4012E000200D1816186D78E4
:101DD00086F84B50401C0828F7D308E000200D1867
:101DE00016186D7886F85350401C0828F7D303F86E
:101DF0003D4F9C700549012081F8250070BD000011
:101E00003C060020A4020020D80500201400002079
:101E1000FEE700002DE9F0410E462DED028B96B055
:101E20000F21009107AB06F5E87206F5CA7100F0C4
:101E300083F9052000900F2302AA314607A800F07D
:101E400053F99FED218A4FF0FF384546002402AF39
:101E500006EB8400D0ED4B0A07EB840090ED000AFE
:101E600000F0ACF9B4EEC80AF1EE10FA02D2B0EE0E
:101E7000408A2546641C052CEADB07EB850090EDC3
:101E8000000A06EB8500D0ED500AB7EE002A90ED6F
:101E90004B1A70EE821A61EE211A72EE600A61EE40
:101EA000200AF4EEC00AF1EE10FA0AD2B4EEE10A0A
:101EB000F1EE10FA05D2284616B0BDEC028BBDE853
:101EC000F0814046F8E7000000247449002809DB4F
:101ED00000F01F02012191404009800000F1E02044
:101EE000C0F800117047002809DB00F01F02012133
:101EF00091404009800000F1E020C0F800117047D7
:101F00000907090E002804DB00F1E02080F8001426
:101F1000704700F00F0000F1E02080F8141D7047BA
:101F20000907090E002804DB00F1E02080F8001406
:101F3000704700F00F0000F1E02080F8141D70479A
:101F40000907090E002804DB00F1E02080F80014E6
:101F5000704700F00F0000F1E02080F8141D70477A
:101F60002DED020B019820F0004001909DED000B3B
:101F700002B0704730B500240022074D07E010F88A
:101F8000013B6340EC5C2344DCB2521C92B28A42B7
:101F9000F5D3204630BD0000282400080149086020
:101FA000704700001000002070B5054600244FF473
:101FB0007A7603E0304600F005F8641CAC42F9D3B1
:101FC00070BD000070B500214FF0E0256C690A4A31
:101FD00012685043AB69AA699A42FCD003D2A3EBC2
:101FE0000203194403E0A4EB0206334419441346E8
:101FF0008142F0D370BD000010000020F0B5F3B0B6
:1020000004464FF496722B4928A8FEF72FF91422A4
:10201000294923A8FEF72AF91422274914311EA8BA
:10202000FEF724F93C210FA8FEF752F93C22224981
:1020300028316846FEF71AF900220FAE6F4628AD28
:1020400006EB820090ED000A04EB820080ED650A49
:1020500007EB820191ED000A80ED740A002102EB8A
:10206000820305EB830004EB830300EB810C9CED02
:10207000000A03EB810C8CED000A491C0529F4DBF6
:10208000521C0F2ADCDB002123AB1EAA03EB8100CC
:1020900090ED000A04EB810080ED4B0A02EB810514
:1020A00095ED000A80ED500A491C0529EEDB73B05E
:1020B000F0BD00002827000854280008FFF790FA18
:1020C0000520FFF771FF3A20FFF7FCFB0520FFF723
:1020D0006BFFA520FFF764FBFEF75EF9FFF75EFEDE
:1020E000FEF76AFAF8E70000F0B5059F0025DFED7E
:1020F000111A1BE002EB8506C6ED001A002412E05F
:1021000004EB840C01EB8C0C0CEB850C96ED000AB7
:10211000DCED000A00EB840C9CED001A01EE200AB5
:1021200086ED000A641C9C42EADB6D1CBD42E1DBCB
:10213000F0BD00000000000070B5049D0024F2EE28
:10214000020AB7EE001A1AE000EB8406D6ED001A78
:1021500001EB840696ED000A02EB840671EEC01ACC
:1021600096ED002A03EB840661EEA01A32EE402AB7
:1021700081EE820A30EE010A86ED000A641CAC4250
:10218000E2DB70BD10B500210B4C621892F88E0294
:10219000D071491CC9B21229F7D31320FFF7A2F856
:1021A0001821601CFFF7E6FE60761921601CBDE86F
:1021B0001040FFF7A5BB0000A402002010B530EED0
:1021C000601A81EE200A10EE100A00F091F841EC3E
:1021D000100BFFF7C5FE51EC100B00F003F800EEFA
:1021E000100A10BD21F00042A2F16052B2F5801F2A
:1021F00001F0004328BFD2F17F6C0BD95FEA001CCD
:1022000043EAC20242EB507018BF704728BF20F06B
:1022100001007047B2F5801FBCBF184670474FEAF7
:10222000410C1CF5001F02D2084600F0D7B870B56B
:1022300000F009F800000089FFF7F6BF4FF00040FA
:10224000A0F5800070470EF1020E2EF0030E5EF82E
:10225000046B364205D4012A43EB030515F5001F34
:1022600012D8012841EB010C1CF5001F0CD80ED12F
:102270004FEAD17C15F5001F0CEB4C0C0CF1020C55
:1022800008BF4CEBD37C04E04FF0080C01E04FEAB0
:10229000D37C0CEB4C0526FA05F606F00706B6F1E2
:1022A000040C06D20EEB860CBDE870404CF0010C1D
:1022B0006047DFE80CF0090B02024FF000414FF0DD
:1022C0000000A1F5002170BD19461046012851EB10
:1022D000010418BFD4F5001484BF002001F00041B0
:1022E00070BD0808A0F500114FEA310170470000E9
:1022F00043004FEAD30C4FEA3C0C43401FBF40075A
:102300000CF1605113F0FE4F70471CF0006F03D1C9
:1023100000200CF0004170470CF0004343EA50707D
:1023200010B540EACC0000F00EF800BF00000092AB
:102330004FEA0001FFF7D5BF4FF000414FF000001A
:10234000A1F5002170470EF1020E2EF0030E5EF88B
:10235000044B244204D44FEA4102B2F17F4F11D81A
:102360004FEA4003B3F17F4F0CD80ED14FEAD07C37
:10237000B2F17F4F0CEB4C0C0CF1020C08BF4CEB94
:10238000D17C04E04FF0080C01E04FEAD17C0CEB6B
:102390004C0324FA03F404F00704B4F1040C06D24D
:1023A0000EEB840CBDE810404CF0010C6047DFE8F8
:1023B0000CF0070802024FF00040A0F5800010BDAD
:1023C0000846420018BFD2F1807288BF00F000407A
:1023D00010BD4FF04070E1EE100A7047FF2141EA56
:1023E000D050C00570470000000000000000000051
:1023F0000102030406070809A0860100400D03003E
:10240000801A060000350C0040420F0080841E0038
:1024100000093D0000127A000024F40000366E012D
:102420000048E801006CDC02005EBCE2613FDD8335
:10243000C29C7E20A3FD1F419DC3217FFCA2401EA4
:102440005F01E3BD3E6082DC23079FC1421CFEA00A
:10245000E1BF5D0380DE3C62BEE0025CDF81633D84
:102460007C22C09E1D43A1FF4618FAA427799BC574
:1024700084DA3866E5BB5907DB856739BAE4065864
:102480001947A5FB7826C49A653BD987045AB8E654
:10249000A7F91B45C6987A24F8A6441A99C7257B44
:1024A0003A6486D85B05E7B98CD2306EEDB3510F34
:1024B0004E10F2AC2F7193CD114FADF3702ECC9224
:1024C000D38D6F31B2EC0E50AFF1134DCE90722C14
:1024D0006D33D18F0C52B0EE326C8ED0530DEFB104
:1024E000F0AE4C1291CF2D73CA947628ABF51749F4
:1024F0000856B4EA6937D58B5709EBB536688AD4E4
:1025000095CB2977F4AA4816E9B7550B88D6346AD3
:102510002B7597C94A14F6A8742AC896154BA9F7C3
:10252000B6E80A54D7896B350000C1C081C14001AB
:1025300001C3C003800241C201C6C006800741C773
:102540000005C1C581C4400401CCC00C800D41CD43
:10255000000FC1CF81CE400E000AC1CA81CB400B13
:1025600001C9C009800841C801D8C018801941D9E3
:10257000001BC1DB81DA401A001EC1DE81DF401F73
:1025800001DDC01D801C41DC0014C1D481D5401583
:1025900001D7C017801641D601D2C012801341D393
:1025A0000011C1D181D0401001F0C030803141F123
:1025B0000033C1F381F240320036C1F681F7403773
:1025C00001F5C035803441F4003CC1FC81FD403D43
:1025D00001FFC03F803E41FE01FAC03A803B41FB13
:1025E0000039C1F981F840380028C1E881E9402963
:1025F00001EBC02B802A41EA01EEC02E802F41EF73
:10260000002DC1ED81EC402C01E4C024802541E582
:102610000027C1E781E640260022C1E281E3402392
:1026200001E1C021802041E001A0C060806141A1A2
:102630000063C1A381A240620066C1A681A7406772
:1026400001A5C065806441A4006CC1AC81AD406D42
:1026500001AFC06F806E41AE01AAC06A806B41AB12
:102660000069C1A981A840680078C1B881B94079E2
:1026700001BBC07B807A41BA01BEC07E807F41BF72
:10268000007DC1BD81BC407C01B4C074807541B582
:102690000077C1B781B640760072C1B281B3407392
:1026A00001B1C071807041B00050C1908191405122
:1026B0000193C053805241920196C0568057419772
:1026C0000055C19581944054019CC05C805D419D42
:1026D000005FC19F819E405E005AC19A819B405B12
:1026E0000199C059805841980188C0488049418962
:1026F000004BC18B818A404A004EC18E818F404F72
:10270000018DC04D804C418C0044C1848185404581
:102710000187C047804641860182C0428043418391
:102720000041C1818180404058EEE33C2912983D30
:1027300010A7023EB7B8FB3DB4DA6C3D0CCEE13CCD
:10274000FF010F3D056A0C3D38E27C3C5D139E3D68
:1027500098A59F3C6655063D0E949D3DA0C42A3C1D
:10276000EE13B73C67A79D3EC3B6313DC0A5063DFD
:10277000E70E623EF151EA3DFDE52B3D1EC1FB3CFB
:102780006B7BD83D0F451D3D2F3CE43E7FF8A33DBC
:10279000D334893C6297E63CBD58883D94BB1A28E7
:1027A0008256A83D80D62F3C56EAF53C94B2BF3DF8
:1027B000165FA73DC4FEF13C4634303D84C5D93C8C
:1027C000A859043E82D7463CC27AA23D8346753C56
:1027D000A70E643DDAA7303D59458D3C6B79093E23
:1027E0002937553E15113A3E8AAE923DA085563D99
:1027F0007713093DE22D013D63DEA03DC4E21B3DA0
:1028000013E9963CBFC4C83CA02EA53CF67F053D0D
:102810005E7EE33C48A0893D26F9B93CF7861B3E25
:10282000F2786F3D4ED98D3DCD9D083D1B53CA3C7E
:102830005F88763E79F6BE3DC8D6243D94BB1A2803
:10284000A10C843DD7F73B3DD11B1A3DA0DA4D3C8E
:1028500094BB1A28F98F8A40E696813FA0D69D3F07
:10286000C299124073DFE93F31B80F3E8739933D7B
:102870001312B03EC7C5203F244A9C3E00002041B1
:102880000000A0400000A04000001B4300004842A0
:102890000000C842000020410000A0410000C842E2
:1028A0000000F0420000F04100E044450000A0407C
:1028B0000000A04000000000000000000000000038
:1028C00000000000378919404260894085EBB5411E
:1028D0007B146E3F713D8A3F0AD7A33E9A99993E79
:1028E000666686403333734000002040000020417C
:1028F000000008410000A040CDCC4C3F33331340D2
:102900000000803F0000164300002040CDCCCC3DAD
:102910009A99193ECDCC4C3ECDCC4C3D3C2900087B
:102920000000002014000000C80100085029000821
:1029300014000020D40C0000E40100081000000086
:10294000010000000000000000093D000000000040
:040000050800018D61
:00000001FF
